:020000000EC030
:100004000FB6139513941395139413951394139592
:10001400139409F423950FBE189501E003BF02E081
:1000240009BF01E007BB0FE008BB0FED0DBF7894DB
:1000340034D04F3FE9F306B30870083039F0932FFA
:10004400A0E021D04F73942FA1E01DD00FD036171C
:1000540079F74F73471761F71EF06894C09802C090
:10006400E894C09A1AD04F3FE9F7E2CF80E005D078
:10007400642D81E002D0742D0895E199FECF8EBBEA
:10008400E09A4DB20895E199FECFAEBB9DBBE29AD2
:10009400E19A089547E035E00895112422271127B5
:1000A400283008F03DC017331CF4B29BF8CFF8CFCA
:1000B4002830B4F5B299FCCF112711318CF5B29BDD
:1000C400FCCF012F1127202E2694322C200E000F56
:1000D400300E12152CF5B299FCCF11275CE04427A1
:1000E40033271215F0F3B29909C08894441F331FC3
:1000F4001315B4F4B29BFCCF112708C00894441F15
:10010400331F13156CF4B299FCCF11275A9549F794
:10011400042F001F331F001F331F4F773F710895B3
:060124004FEF3FEF0895CC
:00000001FF
